:100000000C946F040C948C040C948C040C948C044D
:100010000C948C040C948C040C948C040C94590750
:100020000C948C040C948C040C948C040C948C0410
:100030000C948C040C948C040C948C040C948C0400
:100040000C948C040C948C040C9411060C948C0469
:100050000C948C040C948C040C948C040C948C04E0
:100060000C948C040C948C04204B422F73000D0ACA
:1000700000746D3A2074657374206D6F6465202080
:1000800020200074703A2075647020706F727420A4
:10009000202020200074693A206970206164647215
:1000A0006573732020200074743A207061636B655F
:1000B000742074797065202000746C3A207061633C
:1000C0006B6574206C656E2020200066633A2066A4
:1000D0006C6F7720636F6E74726F6C200066643A89
:1000E0002066756C6C206475706C65782020006DDE
:1000F0003A206D616320616464726573732020200F
:10010000001A11AFA047110000EA05FDFFC0A802C8
:10011000DE901A0020202B7265713D0020763D0094
:1001200020643D00206E3D005D204552523A005D46
:10013000206F6B005B52583A005B54583A003F3FC7
:10014000204552523A00636D643D0046545064614C
:10015000740046545063746C00424F4F5450430037
:10016000424F4F545053002C61636B3D002C73651C
:10017000713D002C666C6167733D005B5443503ADF
:10018000005B5544503A002C55445020002C5443F9
:100190005020002C49434D50005B4950343A0052E6
:1001A00045504C0052455120005B4152503A003FAF
:1001B0000074780072782070696F00727820706C1B
:1001C0006970626F7800636E742020627974657361
:1001D00020202020657272202064726F702072616E
:1001E00074650D0A00F5018F1185103A11B9108C54
:1001F000115B12A110656E6332386A363000706987
:100200006F3A20657869740D0A004552524F523A90
:1002100000207265763D0020666C6167733D003A90
:10022000206F6B21206D61633D0070696F3A20691A
:100230006E69743A2000E5015544503A200041525D
:1002400050205245504C59210D0A00415250205225
:1002500045513A2049503D004552524F523D0020F1
:100260006E3D00763D0070696F2074783A2000453D
:1002700052524F523D00206E3D00763D0070696F36
:100280002072783A20005B50494F5F544553545DCB
:10029000206F66660D0A005B50494F5F544553540A
:1002A0005D206F6E0D0A006F6666006F6E005B4129
:1002B00055544F5D2000544F54414C204552524FED
:1002C000525320004552523A20646174612040002C
:1002D0004552523A20706B7420747970650D0A0093
:1002E0004552523A20737263206D61630D0A0045D6
:1002F00052523A20647374206D61630D0A004552B6
:10030000523A2073697A650D0A005B50425F54458A
:1003100053545D206F66660D0A005B50425F544582
:1003200053545D206F6E0D0A007265712069676E0F
:100330000D0A005245510D0A0046495253542054AB
:1003400052414E53464552210D0A005B4D414749EB
:10035000435D20726571756573740D0A005B4D41D4
:100360004749435D206F66666C696E650D0A005BE8
:100370004D414749435D206F6E6C696E650D0A0003
:100380005B4252494447455D206F66660D0A004650
:100390004C4F57206F6E0D0A00464C4F57206F662A
:1003A000660D0A004F46464C494E452044524F5078
:1003B0003A2000464952535420494E434F4D494E2E
:1003C00047210D0A005B4252494447455D206F6E4C
:1003D0000D0A004E4F204950563421210D0A004E7F
:1003E0004F204D4147494321210D0A005B425249AC
:1003F0004447455F544553545D206F66660D0A00BF
:100400004F56455257524954453F210D0A005B4211
:1004100052494447455F544553545D206F6E0D0A61
:100420000020202000436F6D6D616E64204B657964
:100430002048656C703A0D0A00436F6D6D616E6403
:100440002048656C703A0D0A006279652E2072654D
:100450007374617274696E672E2E2E0D0A006279B4
:10046000650D0A004855483F0D0A003F3F3F0D0A01
:10047000004552524F520D0A0053594E5441580DE7
:100480000A004F4B0D0A004F4B20284E4545442093
:1004900052455354415254290D0A00524553455474
:1004A0000D0A003E2000436F6D6D616E64204D6F3C
:1004B00064652E20456E746572203C3F3E2B3C7275
:1004C000657475726E3E20666F722068656C702070
:1004D000616E64203C713E2B3C72657475726E3E99
:1004E00020746F206C656176652E0D0A00302E3603
:1004F0002032303135303131370D0A0005079C1973
:10050000F306F1069E19DF06DD06811AC606C4064B
:100510007D1AB306B006751A960693066D1A77060D
:100520007406691A58065506651A45064206611A88
:1005300031062F063E1A13061006F819F705F405C2
:10054000F819DE05DB05C019C405C105C019A805E9
:10055000A505A01990058D05C0197B057805F8192A
:10056000680500000000000074657374206D6F64FE
:1005700065205B307C315D00746D007465737420A0
:1005800055445020706F7274203C6E3E00747000B1
:1005900074657374204950206164647265737320BC
:1005A0003C69703E00746900746573742070616307
:1005B0006B6574206574682074797065203C6E3EAC
:1005C0000074740074657374207061636B657420CB
:1005D0006C656E677468203C6E3E00746C007365D9
:1005E0007420666C6F7720636F6E74726F6C205B23
:1005F0006F6E5D006663007365742066756C6C20B9
:100600006475706C65206D6F6465205B6F6E5D0056
:100610006664006D61632061646472657373206F4A
:100620006620646576696365203C6D61633E006D9C
:10063000007265736574207374617469737469639F
:10064000730073720064756D7020737461746973E4
:1006500074696373007364007265736574207061FC
:1006600072616D657465727320746F206465666174
:10067000756C74007072006C6F61642070617261DF
:100680006D65746572732066726F6D2045455052BA
:100690004F4D00706C007361766520706172616D02
:1006A000657465727320746F20454550524F4D003C
:1006B0007073007072696E7420706172616D657420
:1006C0006572730070007072696E74206669726D75
:1006D000776172652076657273696F6E007600735C
:1006E0006F667420726573657420646576696365EE
:1006F0000072007175697420636F6D6D616E6420A6
:100700006D6F64650071004F46460D0A004F4E0D37
:100710000A00564552424F53453A2000318F1A3253
:100720000832921A1B08338B1A070834871AF40709
:1007300073B61AE40753B41AD307769E1ABD07702E
:100740009B1A9C0750981A720761961A530700006B
:10075000000000746F67676C65206175746F2073AB
:10076000656E642028706274657374206D6F6465B3
:10077000290073656E642061207465737420706154
:10078000636B6574202873696C656E74292028700A
:100790006274657374206D6F6465290073656E649F
:1007A00020612074657374207061636B6574202808
:1007B000706274657374206D6F64652900746F676F
:1007C000676C6520766572626F7365206F757470F3
:1007D00075740072657365742073746174697374E1
:1007E0006963730064756D702073746174697374E8
:1007F00069637300656E746572205042207465737E
:1008000074206D6F646500656E7465722050494F89
:100810002074657374206D6F646500656E74657215
:10082000206272696467652074657374206D6F64FB
:100830006500656E74657220627269646765206D1B
:100840006F646500726573657474696E672E2E2E11
:100850000D0A005072657373203C72657475726E78
:100860003E20746F20656E74657220636F6D6D61DC
:100870006E64206D6F6465206F72203C3F3E206681
:100880006F72206B65792068656C700D0A00627963
:10089000206C616C6C6166612028687474703A2FFA
:1008A0002F7777772E6C616C6C6166612E64652F93
:1008B000626C6F67290D0A0D0A000D0A57656C639B
:1008C0006F6D6520746F20706C6970626F78203076
:1008D0002E362032303135303131370D0A001124B7
:1008E0001FBECFEFD8E0DEBFCDBF11E0A0E0B1E08A
:1008F000ECEFF6E302C005900D92A034B107D9F7F2
:1009000027E0A0E4B1E001C01D92AB3EB207E1F7E1
:100910000E94B81A0C94F51A0C940000F89484B74D
:10092000877F84BFE0E6F0E0808188618083108269
:10093000789408958A3010F4805D0895895C089554
:100940001F93CF93DF93182FEB0182958F700E9436
:100950009A048883812F8F700E949A048983DF9183
:10096000CF911F9108951F93CF93DF93182FEB0121
:10097000892F0E94A004BE016E5F7F4F812FDF91FF
:10098000CF911F910C94A004CF92DF92EF92FF922F
:10099000CF93DF936B017C01EA01BA01C7010E948A
:1009A000B304BE016C5F7F4FC601DF91CF91FF9012
:1009B000EF90DF90CF900C94B304FB0164E60E94AB
:1009C000341B805D8083892F6AE00E94341B805D28
:1009D0008183905D92830895AF92BF92CF92DF9210
:1009E000EF92FF920F931F93CF93DF93EA01B22E02
:1009F000E22FF0E03197CE0FDF1F021708F42196A7
:100A000010E02EE2A22E3AE0C32ED12CE12CF12CE4
:100A10001B1579F0101302C0A8822197A701960137
:100A20000E94401B605D68832197B901CA011F5F66
:100A3000EFCFDF91CF911F910F91FF90EF90DF905B
:100A4000CF90BF90AF900895FB019FE9980F96302B
:100A500010F4875509C09FEB980F963010F4875318
:100A600003C080538A3018F4808381E0089580E0C9
:100A70000895EF92FF920F931F93CF93DF931F92EE
:100A8000CDB7DEB77C018B01BE016F5F7F4FFC01EC
:100A900080810E942405811102C080E011C08981FB
:100AA0008295807F8983B801F70181810E942405A6
:100AB000882399F3F80180819981892B808381E0D3
:100AC0000F90DF91CF911F910F91FF90EF900895BC
:100AD000EF92FF920F931F93CF93DF9300D0CDB788
:100AE000DEB78C017B01BE016E5F7F4F0E9439052E
:100AF000811102C080E013C0BE016F5F7F4FC8014B
:100B000002960E9439058823A9F38A8190E0982FE4
:100B100088272981822BF7019183808381E00F90C0
:100B20000F90DF91CF911F910F91FF90EF9008955B
:100B3000EF92FF920F931F93CF93DF9300D000D0DB
:100B4000CDB7DEB77C018B01BE016C5F7F4F0E9489
:100B50003905811102C080E02EC0BE016D5F7F4F5C
:100B6000C70102960E9439058823A9F3BE016E5F72
:100B70007F4FC70104960E943905882361F3BE01A7
:100B80006F5F7F4FC70106960E943905882319F3CE
:100B90002C818B8190E0A0E0B0E0DC0199278827D0
:100BA000B22B2981822B2A81922BF8018083918399
:100BB000A283B38381E00F900F900F900F90DF918D
:100BC000CF911F910F91FF90EF900895FC0180E06D
:100BD00020E0919190539A3048F43AE0239F900D91
:100BE0001124292F8F5F8330A1F702C0882311F0D1
:100BF000FB0120830895F894E1ECF0E0108210925C
:100C0000C50080E18093C40088E9808386E88093F2
:100C1000C20078941092420110924101109240015A
:100C200008951F920F920FB60F9211248F93EF9396
:100C3000FF938091C600E0914101F0E0ED5BFE4F33
:100C40008083809141018F5F8093410180914101B8
:100C5000803111F410924101809140018F5F8093A7
:100C60004001FF91EF918F910F900FBE0F901F9059
:100C70001895209142019091410181E0291301C012
:100C800080E0089590914201809141019817D1F33D
:100C9000F894E0914201F0E0ED5BFE4F808190918D
:100CA00042019F5F9093420190914201903111F473
:100CB000109242019091400191509093400178949C
:100CC00008959091C00095FFFCCF8093C6000895D1
:100CD000CF93DF93EC01FE018491882321F00E94E1
:100CE00061062196F8CFDF91CF910895CF93DF93DE
:100CF000EC018991882319F00E946106FACFDF91F7
:100D0000CF910895EF92FF921F93CF93DF931F929D
:100D1000CDB7DEB7182F7C018E2D811B861740F4CE
:100D2000F70181917F0169830E9461066981F4CF97
:100D30000F90DF91CF911F91FF90EF9008958EE675
:100D400090E00C94680680E20C9461060F93609129
:100D50005F0170916001809161019091620104E0F6
:100D60002AE043E551E00E94EC0480E280935E01BA
:100D70006CE083E591E00F910C9482060F9304E000
:100D80002AE043E551E00E94EC0480E280935E019A
:100D90006CE083E591E00F910C9482060F93BC0107
:100DA00080E090E002E026E043E551E00E94EC04A0
:100DB00067E083E591E00E94820688E690E00F916B
:100DC0000C9468060F93DC01CB01009721E0A20789
:100DD000B10538F021E22093530164E571E0CD01C3
:100DE0000BC0803127E29207A105B10540F02EE348
:100DF0002093530164E571E00E94B3040BC02BE221
:100E00002093530104E024E044E551E0BC01CD010E
:100E10000E94EC0465E083E591E00F910C9482065A
:100E200063E571E00E94A00462E083E591E00C9428
:100E3000820663E571E00E94B30464E083E591E01B
:100E40000C94820643E551E00E94C40468E083E507
:100E500091E00C948206F89482E08093B000809335
:100E6000B10097EC9093B3001092B20080937000A1
:100E70001092800083E08093810010928200109293
:100E80008500109284001092660110926501109204
:100E900064011092630110925F0110926001109240
:100EA00061011092620110926801109267017894BA
:100EB00008951F920F920FB60F9211242F938F93C4
:100EC0009F93AF93BF9380916501909166010196C6
:100ED000909366018093650180915F01909160011C
:100EE000A0916101B09162010196A11DB11D809395
:100EF0005F0190936001A0936101B09362018091C2
:100F00006701909168010196883E23E0920729F0DD
:100F100090936801809367010DC010926801109250
:100F2000670180916301909164010196909364013F
:100F300080936301BF91AF919F918F912F910F90FB
:100F40000FBE0F901F9018951092640110926301CC
:100F5000209163013091640128173907C8F308957F
:100F60001092660110926501209165013091660131
:100F700028173907C8F30895FB013097A9F0DC0161
:100F800020EA36E841E050E00E94621B9F0140E009
:100F900050E0E2E0220F331F441F551FEA95D1F7BE
:100FA0000E94401BC901089580E090E0089587B138
:100FB0008F6387B98AB1806C8AB9089587B1807CC4
:100FC00087B98AB18F738AB9089553985B9A21982B
:100FD000299A549A5C9855985D9A209A289A0C946C
:100FE000DE0728988A95F1F7289A089510926601ED
:100FF000109265012091000130910101409165013D
:10100000509166014217530780F499B195FB9927D7
:1010100090F9882319F0992319F00AC0992341F017
:101020001999ECCF862F83600895862F82600895EA
:1010300081E00895909384018093830170938201ED
:10104000609381015093800140937F0130937E0132
:1010500020937D010E94DE075C98089589B123B139
:1010600099B1907283FB882780F921FD82609111EC
:101070008460089581E00E94F10780915F01909162
:101080006001A0916101B091620180937901909318
:101090007A01A0937B01B0937C0108955F926F92D7
:1010A0007F928F929F92AF92BF92CF92DF92EF92F8
:1010B000FF920F931F93CF93DF9300D01F92CDB772
:1010C000DEB710926901199904C010926A0180E09C
:1010D00091C24D99FACF86B159B0952D907C592E79
:1010E0008F73582A1A821982E2E25E1619F0F4E42C
:1010F0005F1215C060917D0170917E01E0918301C6
:10110000F0918401AE014F5F5F4F80917F0190911C
:1011100080010995813019F080936A016BC2C090FB
:101120005F01D0906001E0906101F0906201109247
:101130008500109284005C9A82E2581681F0851531
:1011400028F091E1591609F488C0E8C1E3E35E167E
:1011500009F478C1F4E45F1609F4E9C0DFC109813C
:101160001A8160E281E00E94F607282F813009F0A1
:10117000CEC10E94D70796B1812F8F73907C892BA7
:1011800088B999B1812F807C9F73892B8BB95C982A
:1011900060E380E00E94F607282F813009F0B7C194
:1011A00086B1807C902F9F73892B88B989B18F730A
:1011B000902F907C892B8BB95C9A00FF02C00F5F47
:1011C0001F4F48019694879460907F017090800132
:1011D000A12CB12C8501000F111FA814B904A1F195
:1011E00060E481E00E94F607282F813091F5F30139
:1011F000808126B1982F9F73207C922B98B999B14A
:10120000807C9F73892B8BB95C9860E480E00E949E
:10121000F607282F813019F00F5F1F4F1AC0F30116
:10122000818126B1982F9F73207C922B98B999B118
:10123000807C9F73892B8BB95C9AFFEFAF1ABF0A32
:1012400082E0680E711CC6CF60E581E00E94F6075F
:10125000282F2B830E94DE07F3C060E281E00E940A
:10126000F607282F813009F052C116B109B15C98F8
:1012700060E380E00E94F607282F813009F047C123
:1012800096B189B15C9A302F307C1F73312B632E5D
:10129000712C762C6624807C9F73892B682A809120
:1012A0007D0190917E018615970508F433C160FE9B
:1012B00003C09FEF691A790A7694679480907F0142
:1012C00090908001A12CB12C8501000F111FA61454
:1012D000B70409F426C160E481E02B830E94F6077D
:1012E0002B81813011F596B189B1807C9F73892B58
:1012F000F40180835C9860E480E02B830E94F60711
:101300002B81813019F00F5F1F4F0FC096B189B14B
:10131000807C9F73892BF40181835C9AFFEFAF1A65
:10132000BF0A82E0880E911CCFCF282FFAC0098116
:101330001A8160E281E00E94F607282F813009F0CF
:10134000E6C00E94D70796B1812F8F73907C892BBE
:1013500088B999B1812F807C9F73892B8BB95C9858
:1013600060E380E00E94F607282F813009F0CFC0AB
:1013700086B1807C902F9F73892B88B989B18F7338
:10138000902F907C892B8BB95C9A60E481E00E945D
:10139000F607282F813009F0BAC00F5F1F4F16954E
:1013A0000795E0917F01F0918001F8945C98A12C61
:1013B000B12C46E0A016B10699F0842F8A95F1F77A
:1013C000808136B1982F9F73307C932B98B999B157
:1013D000807C9F73892B8BB94D9B04C01999FCCFDE
:1013E00078941BC0842F8A95F1F7818136B1982FAC
:1013F0009F73307C932B98B999B1807C9F73892B14
:101400008BB94D9903C01999FCCFEACF32969FEF63
:10141000A91AB90ACFCF199BE3CF4D99FCCF5C9A9B
:101420004D9903C01999FCCFDBCFA016B10608F483
:1014300022E45C982B830E94DE078501000F111FB8
:101440002B816FC060E281E00E94F607282F813077
:1014500009F05DC016B109B15C9860E380E00E94BC
:10146000F607282F813009F052C046B139B1802FDC
:10147000807C1F73812B90E0982F8827307C4F73DE
:10148000342B832B40917D0150917E0148175907E1
:1014900008F440C001969695879540917F01309160
:1014A0008001F8945C9AE42FF32F00E010E0081715
:1014B000190721F478941BC0199BFCCF4D9BFCCFDE
:1014C00046B139B1307C4F73342B30834D9B03C010
:1014D0001999FCCFEFCF46B139B1307C4F73342B23
:1014E00031830F5F1F4F3296E2CF199BE3CF4D9BA5
:1014F000FCCF5C984D9B03C01999FCCFDBCF08173C
:10150000190708F422E45C9A000F111F0AC000E0DA
:1015100010E007C000E010E025E003C000E010E0AC
:1015200024E0109266011092650180910001909173
:10153000010140916501509166014817590710F467
:101540001999F7CF5C98A0908400B0908500213065
:1015500089F4E1E15E1619F0F3E35F120BC0E0914C
:101560008101F0918201B80180917F019091800109
:101570000995282F5092690120936A0110936E01FA
:1015800000936D01B0927001A0926F01B501C80186
:101590002B830E94BC079093720180937101C092CB
:1015A0007501D0927601E0927701F09278012B815B
:1015B00081E1581631F081E093E3591619F080E08B
:1015C00001C081E080936B0180936C0181110BC09D
:1015D00080917501909176014091790150917A0145
:1015E000841B950B02C080E090E09093740180937F
:1015F0007301822F0F900F900F90DF91CF911F9169
:101600000F91FF90EF90DF90CF90BF90AF909F90A1
:101610008F907F906F905F9008958FEF9FEFEFE630
:10162000F7E021918227282F22952827022E269540
:1016300026952025022E269520252770082E892FF5
:10164000269507942795902D822706942795902517
:10165000822727E0E238F20721F70895CF93DF933E
:101660008FEE90E00E9468068FE697E00E94140CCF
:101670000E949F060E949F06C09176078DED90E024
:101680000E9468068C2F0E9410070E949F06C0913E
:1016900075078BEC90E00E9468068C2F0E94100763
:1016A0000E949F060E949F06C0917707D0917807FD
:1016B00089EB90E00E946806CE010E9419070E9403
:1016C0009F06C0917907D0917A0787EA90E00E943F
:1016D0006806CE010E9419070E949F0685E990E0E6
:1016E0000E9468068BE797E00E948B0C0E949F0681
:1016F000C0917F07D091800783E890E00E94680640
:10170000CE010E9419070E949F06C091810781E7C0
:1017100090E00E9468068C2F0E941007DF91CF9105
:101720000C949F06F99911C043E150E062E070E02B
:101730008FE697E00E94171B0E940D0BBC0180E012
:1017400090E00E942F1B80E0089581E00895AFE6AD
:10175000B7E0E1E0F1E084918D93319681E0E431EE
:10176000F807C9F70895CF93DF93F99916C043E1BD
:1017700050E062E070E08FE697E00E94011B80E09D
:1017800090E00E94111BEC010E940D0BC817D907B5
:1017900031F00E94A70B82E003C081E001C080E02D
:1017A000DF91CF9108950E94B30B81110C94A70B88
:1017B0000895FB0120E030E0DC014D91CD01419323
:1017C0002F5F3F4F26303105B9F70895FB0120E028
:1017D00030E0DC014D91CD0141932F5F3F4F24302C
:1017E0003105B9F70895FC01808190E0982F882792
:1017F0002181822B0895FC01708361830895FC018F
:1018000020816181862F90E0A0E0B0E077276627F5
:10181000922B2381622B2281722B0895FC0170830D
:1018200061835283438308950F931F93CF93DF9374
:101830008C01CEE1D1E0BE01F80181918F010E94BF
:10184000A0042396F1E0C033DF07A9F78EE191E011
:10185000DF91CF911F910F910C947606CF92DF927A
:10186000EF92FF920F931F93CF93DF931F92CDB709
:10187000DEB77C016B0100E010E0BE016F5F7F4FBF
:10188000C7010E94E605882371F090E00196E80EFA
:10189000F91E8981F60181936F010F5F1F4F04309C
:1018A000110559F781E00F90DF91CF911F910F91B2
:1018B000FF90EF90DF90CF900895CF92DF92EF925C
:1018C000FF920F931F93CF93DF931F92CDB7DEB795
:1018D0007C016B0100E010E0BE016F5F7F4FC7012C
:1018E0000E943905882369F083E0E80EF11C8981A4
:1018F000F60181936F010F5F1F4F0630110561F7ED
:1019000081E00F90DF91CF911F910F91FF90EF90A9
:10191000DF90CF9008950F931F93CF93DF938C01A7
:10192000C0E3D1E0BE01F80181918F010E94DD0486
:101930002496F1E0C034DF07A9F780E391E0DF915E
:10194000CF911F910F910C947606FB0120E030E0BF
:10195000DC015D91CD014191541307C02F5F3F4FD2
:1019600026303105A9F781E0089580E00895FB0154
:1019700020E030E0DC015D91CD014191541307C0BE
:101980002F5F3F4F24303105A9F781E0089580E0B3
:1019900008950F931F93CF93DF93EC016C31710582
:1019A000A0F00E94F30B8C01CE0102960E94F30B73
:1019B0003C812D810130110541F48115984029F4B5
:1019C000363019F481E0243009F080E0DF91CF91C6
:1019D0001F910F910895AF92BF92CF92DF92EF9235
:1019E000FF920F931F93CF93DF93EC016B015A018A
:1019F00062E070E006960E94FB0B7E0188E0E80E34
:101A0000F11CBE016E5E7F4FC7010E94D90B8E0193
:101A1000025F1F4FBE01685E7F4FC8010E94E60B48
:101A2000B701C6010E94D90BB801C501DF91CF9162
:101A30001F910F91FF90EF90DF90CF90BF90AF90EC
:101A40000C94E60BCF93DF93EC018334910519F4EA
:101A500080E691E005C08434910531F489E591E098
:101A6000DF91CF910C94680680E20E946106CE015E
:101A70000E94190780E2DF91CF910C946106CF9309
:101A8000DF93EC018531910519F482E591E005C001
:101A90008431910531F48BE491E0DF91CF910C9486
:101AA000680680E20E946106CE010E94190780E26A
:101AB000DF91CF910C946106EF92FF920F931F93E9
:101AC000CF93DF9300D000D0CDB7DEB77C018B0180
:101AD0008BE50E946106B80180E090E004E024E01C
:101AE000AE014F5F5F4F0E94EC0464E0CE010196AF
:101AF0000E9482068CE20E946106C7010C960E9439
:101B0000F30B0E9419078CE20E946106C70106963A
:101B10000E94140C8EE30E946106C7010E94140CFF
:101B20008DE50E94610680E20E9461060F900F9091
:101B30000F900F90DF91CF911F910F91FF90EF9039
:101B40000895CF93DF93EC0189EA91E00E94680643
:101B5000CE0106960E94F30B8130910519F484EAB8
:101B600091E005C08230910529F48FE991E00E944F
:101B7000680602C00E9419078CE20E94610688E292
:101B80000E946106CE0108960E94140C8CE20E940D
:101B90006106CE010E960E948B0C89E20E946106BE
:101BA0008EE30E94610688E20E946106CE014296A1
:101BB0000E94140C8CE20E946106CE0148960E949D
:101BC0008B0C89E20E9461068DE50E94610680E22D
:101BD000DF91CF910C9461061F93CF93DF93EC01BB
:101BE00089E991E00E9468068A8190E0982F882711
:101BF0002B81822B0E9419071985113019F483E972
:101C000091E004C0163029F48DE891E00E94680646
:101C10000CC0113119F487E891E0F8CF8CE20E94F2
:101C20006106812F90E00E9419078CE20E946106F4
:101C3000CE010C960E948B0C8EE30E946106CE01B1
:101C400040960E948B0C8DE50E94610680E2DF9138
:101C5000CF911F910C946106CF92DF92EF92FF9289
:101C6000CF93DF93FC0120812F70220F220F7C0184
:101C7000E20EF11C81858131B9F481E891E00E9486
:101C80006806C7010E94F30B6C01C70102960E940F
:101C9000F30BEC01C6010E94220D8EE30E94610647
:101CA000CE010E94220D40C0863009F049C08BE76A
:101CB00091E00E946806C7010E94F30BEC01C70186
:101CC00002960E94F30B6C01CE010E943F0D8EE341
:101CD0000E946106C6010E943F0DC7010C960E943A
:101CE000F30B6C0183E791E00E946806C6019170D6
:101CF0000E9419078DE691E00E946806C7010496CC
:101D00000E94FF0B0E942207C4FE0EC0C701089666
:101D10000E94FF0B6B017C0187E691E00E94680640
:101D2000C701B6010E9422078DE50E94610680E28C
:101D3000DF91CF91FF90EF90DF90CF900C946106F0
:101D4000DF91CF91FF90EF90DF90CF9008950F93A8
:101D50001F93CF93DF938C010E945C0DE8012E96B8
:101D6000C8010C960E94F30B863028E0920739F4E4
:101D7000CE01DF91CF911F910F910C94A10D811590
:101D8000984051F4CE010E94EC0DCE01DF91CF912D
:101D90001F910F910C942C0EDF91CF911F910F91F9
:101DA0000895EF92FF920F931F93CF93DF9300D08C
:101DB00000D0CDB7DEB77C010E94A606F7011081E6
:101DC000123241F018F4113139F404C0133311F018
:101DD000143411F481E001C080E0F7010181811128
:101DE0000FC086E491E00E946806812F0E941007D0
:101DF0008EE391E00E946806802F0E9410075DC06C
:101E0000F7018281882319F089E391E002C084E31D
:101E100091E00E946806812F0E941007013029F48A
:101E20008FE291E00E94680607C088E291E00E947C
:101E30006806802F0E94100784E291E00E946806E5
:101E4000F7016481758180E090E004E024E0AE0158
:101E50004F5F5F4F0E94EC0464E0CE0101960E9448
:101E6000820680E291E00E946806F7016681778130
:101E700080E090E024E0AE014F5F5F4F0E94EC04F1
:101E800064E0CE0101960E9482068CE191E00E94FE
:101E90006806F701808591850E94CE06F701828150
:101EA00081110BC084E191E00E946806F701628510
:101EB000738580E090E00E94E2060E949F060F90EA
:101EC0000F900F900F90DF91CF911F910F91FF9086
:101ED000EF900895FF920F931F93CF93DF93F82E07
:101EE000082F10E08CE0F89EE0011124CE57D84F67
:101EF0008C819D810E9419070E94A30668817981C7
:101F00008A819B810E9422070E94A3068E819F8165
:101F10000E9419070E94A306888599850E941907C7
:101F20000E94A3068A859B850E94CE060E94A30676
:101F300083E08F1540F0F801EE0FFF1FEA5EFE4FC1
:101F40008081918102C08FEA91E00E946806DF9152
:101F5000CF911F910F91FF900C949F06E2E8F7E05C
:101F600010821182128213821582148217821682C5
:101F700011861086138612863C9687E0E23BF807AE
:101F800079F708950F931F939CE0899FF001112426
:101F9000EE57F84F84819581019695838483008163
:101FA000118122813381060F171F211D311D0083EE
:101FB000118322833383828593858417950710F4D8
:101FC000538742871F910F91089586EC91E00E94FC
:101FD000680680E00E946A0F81E00E946A0F82E03A
:101FE0000E946A0F83E00C946A0FCF93DF93D82F7F
:101FF000C62F86EC91E00E946806DD2331F080E078
:102000000E946A0F81E00E946A0FCC2341F082E0B7
:102010000E946A0F83E0DF91CF910C946A0FDF91E9
:10202000CF91089584B18C6284B9249885B1877D5D
:1020300085B92A9A80E58CBD81E08DBD08952A98E6
:102040006F71682B6EBD0DB407FEFDCF4EBD0DB494
:1020500007FEFDCF2A9A08952A982AE32EBD0DB4D3
:1020600007FEFDCFFB01860F971FE817F90739F030
:102070001EBC0DB407FEFDCF2EB52193F6CF2A9AD4
:102080000895CF93C82FC0766C2F70E02091B607CB
:1020900030E06217730781F043E06FE180EA0E944D
:1020A0001F10C093B6074C2F4295469547706FE1BD
:1020B00080E8CF910C941F10CF9108951F93CF9378
:1020C000DF931F92CDB7DEB7182F69830E944110AE
:1020D0004981612F80E40F90DF91CF911F910C9483
:1020E0001F101F93CF93DF931F92CDB7DEB7182F2A
:1020F00079830E945E107981672F81E0810F0F90B4
:10210000DF91CF911F910C945E108FE10E944110DE
:1021100044E06FE180EA0C941F106091B407709165
:10212000B5076150710961158AE1780710F06FEF0A
:1021300079E18CE00E94711040E46EE180E80C943B
:102140001F10811114C08091B307882321F06623EA
:1021500039F082E006C081E0611103C080E001C077
:1021600083E0682F87E70E945E1080E0089581E099
:102170000895CF92DF92EF92FF920F931F93CF9328
:10218000DF9300D000D000D0CDB7DEB77C018B014B
:102190006A016091B4077091B50780E00E947110E8
:1021A000BE016F5F7F4F86E090E00E942C10898116
:1021B0009A819093B5078093B4072B813C8124507A
:1021C0003109F601318320838D8187FD04C00E948F
:1021D0008D1083E00FC00217130718F08901D12C6E
:1021E00002C082E0D82EB701C8010E942C100E94C4
:1021F0008D108D2D26960FB6F894DEBF0FBECDBF85
:10220000DF91CF911F910F91FF90EF90DF90CF90D2
:1022100008952A98982F9F719EBD0DB407FEFDCF9B
:1022200087FD02C01EBC05C01EBC0DB407FEFDCF5D
:10223000F9CF0DB407FEFDCF8EB52A9A0895CF933E
:10224000C82F0E9441108C2FCF910C940911CF936D
:10225000DF93EB01682F84ED0E945E10BE0186EDD6
:102260000E9471108AEE0E941F1180FDFBCFDF914A
:10227000CF910895EF92FF921F93CF93DF931F9218
:10228000CDB7DEB7182F7B0160E07AE182E0998359
:102290000E94711040E060E08AE70E941F102A98B7
:1022A0008AE78EBD99810DB407FEFDCFE12FF92F8E
:1022B000CF018E0D9F1DE817F90731F021912EBD3A
:1022C0000DB407FEFDCFF7CF2A9A8FE10E940911C6
:1022D00083FF10C08CE10E941F1181FFF6CF40E800
:1022E0006FE180E80E941F1040E86FE180EA0E94E1
:1022F0001F10EBCFB701765E86E00E94711048E0B8
:102300006FE180E80E941F1080E00F90DF91CF9175
:102310001F91FF90EF90089589E30C941F11FF9295
:102320000F931F93CF93DF93EC01F62E0E941210B0
:102330002A9A8F2D81708093B3074FEF60E08FEF63
:102340000E941F108FE39FE10197F1F700C000008A
:102350000FEF1FE08DE10E940911811107C00150AC
:10236000110901151105B1F781E09FC01092B50761
:102370001092B40760E070E088E00E94711060E0A5
:1023800070E08CE00E9471106FEF79E18AE00E94AA
:10239000711060E07AE184E00E9471106FEF7FE1DC
:1023A00086E00E947110F2FE02C061EA01C060EA9C
:1023B00088E30E945E106FE370E388E20E94711070
:1023C00069EF77EF80E30E9471106DE080EC0E946E
:1023D0005E1060E081EC0E945E101091B307111155
:1023E00002C062E301C063E382EC0E945E1011232D
:1023F00039F065E184EC0E945E1062E170E006C095
:1024000062E184EC0E945E1062E17CE086EC0E9456
:1024100071106EEE75E08AEC0E947110112341F08C
:1024200060E071E080E00E94271160E070E007C08A
:1024300060E070E080E00E94271160E071E080E1E0
:102440000E94271160ED77E088E70E94711082E713
:102450000E941F11863008F08F5F8093B207688159
:1024600084EE0E945E10698185EE0E945E106A8192
:1024700082EE0E945E106B8183EE0E945E106C8182
:1024800080EE0E945E106D8181EE0E945E108FE1F1
:102490000E94411040EC6BE180E80E941F1044E074
:1024A0006FE180E80E941F1080E0DF91CF911F91C3
:1024B0000F91FF900895CF93DF93EB01882359F09C
:1024C0008130F1F461E184ED0E945E1061E082ED03
:1024D0000E945E1003C08091B2070FC08AEE0E9476
:1024E0001F1180FDFBCF60E082ED0E945E1089ED40
:1024F0000E941F1182FB882780F9888380E002C038
:10250000188281E0DF91CF910895811104C010926B
:10251000B90781E0089580E00895EF92FF920F934C
:102520001F93CF93DF931F92CDB7DEB78C01F62EAA
:10253000E091B907F0E0EE0FFF1FEA5CFD4F8591D7
:1025400094919093B8078093B7070E94A6068AE2F9
:1025500092E00E946806E091B707F091B807859174
:1025600094910E946806E091B707F091B8073296FF
:10257000259134916F2DC801F9010995E82E81113B
:1025800024C08FE192E00E946806C8010E94140CEA
:1025900087E192E00E9468068F2D0E941007E0916B
:1025A000B707F091B8073C9625913491BE016F5F53
:1025B0007F4F80E0F9010995E82E81110DC081E17E
:1025C00092E00E946806898105C08AE092E00E943C
:1025D00068068E2D0E9410070E949F068E2D0F9078
:1025E000DF91CF911F910F91FF90EF9008950E947E
:1025F000A6068EEF91E00E946806E091B707F09181
:10260000B807349685919491FC010994E091B7073D
:10261000F091B807369625913491F9010994E0912B
:10262000B707F091B807389625913491F9010994CC
:10263000E091B707F091B8073A9685919491FC0123
:102640000994E091B707F091B8073C962591349131
:10265000F9010994E091B707F091B8073E962591EA
:102660003491F901099480917507811102C084E0C9
:1026700001C08CE090917607911181600895FF92DE
:102680000F931F93CF93DF93EC011092850010926C
:102690008400AC016AEE75E085E891E00E940F13BA
:1026A000F82E60918400709185000990D881C02D2A
:1026B000CE010E94BC078C01F11006C0AC01BE0126
:1026C00082E00E94C20F0AC02091A0073091A107AA
:1026D0002F5F3F4F3093A1072093A0078091E90718
:1026E000882301F10E94A6068DE792E00E94680609
:1026F000F1100FC08AE792E00E946806C8010E94AC
:10270000CE0686E792E00E946806CE010E94190775
:1027100007C08FE692E00E9468068F2D0E94100786
:102720000E949F068F2DDF91CF911F910F91FF90F7
:102730000895FF920F931F93CF93DF93EC011092B4
:10274000850010928400BC0185E891E00E94061388
:10275000F82E6091840070918500CE010E94BC0724
:102760008C01F11006C0AC01BE0183E00E94C20FD3
:102770000AC02091AC073091AD072F5F3F4F3093D7
:10278000AD072093AC078091E907882301F10E94EF
:10279000A60686E692E00E946806F1100FC083E666
:1027A00092E00E946806C8010E94CE068FE592E082
:1027B0000E946806CE010E94190707C088E592E0D2
:1027C0000E9468068F2D0E9410070E949F068F2D81
:1027D000DF91CF911F910F91FF900895CF93DF93D9
:1027E000EC0181E991E00E94F30B8630984009F0FA
:1027F0004FC0CF30D10508F44BC0BE016E507109F7
:1028000083E991E00E94C90C882309F43FC089E95B
:1028100091E00E94F30B0197C9F58091E9078823A5
:1028200061F00E94A6068BE492E00E9468068BEAA3
:1028300091E00E948B0C0E949F066BE777E08BEA89
:1028400091E00E94B70C882309F14BE757E06FE64F
:1028500077E083E991E00E94EB0C65E871E080E1AC
:1028600091E00E94D90B6BE871E08FE697E00E943F
:10287000D90BCE010E9499138091E907882331F08A
:102880000E94A6068EE392E00E94680681E001C0E5
:1028900080E0DF91CF910895CF92DF92EF92FF9287
:1028A0000F931F93CF93DF93C0919301CF70CC0F01
:1028B000CC0FD0E0CD56DE4F8E010E5F1F4FC8010A
:1028C0000E94F30B7C0163EA71E08BE797E00E94C2
:1028D000B70C8823E1F180917F0790918007E8167B
:1028E000F906A9F58091E907882359F00E94A60608
:1028F00088E392E00E94680688850E9410070E9483
:102900009F0663EA71E08FE991E00E94E60B6FE9B0
:1029100071E08BE797E00E94E60BCE010E94F30B7B
:102920006C01B701CE010E94FB0BB601C8010E94E9
:10293000FB0B65E871E08BE891E00E94D90B6BE836
:1029400071E08FE697E00E94D90B81E001C080E042
:10295000DF91CF911F910F91FF90EF90DF90CF907B
:1029600008951F93CF93DF9300D0CDB7DEB70E94B9
:10297000A60687E992E00E9468060E943313682F3A
:102980008FE697E00E948D120E94AE0F10E08091BA
:10299000EA07833059F50E946418182F81FD26C07C
:1029A0000E941813882399F3CE0101960E943F13C9
:1029B000811111C089819A810E94EE138111E7CFA4
:1029C00089819A810E944C14882309F389819A8114
:1029D0000E949913DCCF2091A0073091A1072F5FAF
:1029E0003F4F3093A1072093A007D1CF61E080E053
:1029F0000E94F50F0E94F7120E94A60686E892E058
:102A00000E946806812F0F900F90DF91CF911F9148
:102A10000895CF930E944E08C82F882359F1813022
:102A2000A9F4409171015091720160916D01709112
:102A30006E0180916C010E94C20F8091E90788238A
:102A4000D9F089E691E00E94D10E16C089E691E0A6
:102A50000E94D10EE0916C018CE0E89FF0011124FE
:102A6000EE57F84F268137812F5F3F4F37832683FC
:102A70008C2F03C080E001C081E0CF910895CF92F8
:102A8000DF92EF92FF920F931F93CF93DF938C010E
:102A90007B0180917707909178076817790739F063
:102AA0008EEF92E00E946806C1E0D0E002C0C0E074
:102AB000D0E060E171E0C8010E94A50C811105C061
:102AC00021968FEE92E00E9468066FE677E0C801DB
:102AD00006960E94A50C811105C0219680EE92E019
:102AE0000E9468068091790790917A07F801248501
:102AF000291303C09585981729F0219680ED92E05F
:102B00000E9468066701FEE0CF1AD108025F1F4FDE
:102B100076018C2D8E19E114F10491F0F801919158
:102B20008F01981749F084EC92E00E946806C70173
:102B30000E9419070E949F06F1E0EF1AF108E9CF01
:102B4000209759F086EB92E00E946806CE010E9421
:102B500019070E949F0686E001C081E0DF91CF91B6
:102B60001F910F91FF90EF90DF90CF9008950F93FA
:102B70001F93CF93DF93EC018A01809177079091A7
:102B80007807FA01918380836817790720F1BE01E5
:102B900080E191E00E94D90BBE016A5F7F4F8FE612
:102BA00097E00E94D90B8091790790917A079C87D2
:102BB0008D879E01225F3F4FF801808191818C0FAC
:102BC0009D1FF9014E2F421BE817F90711F04193A1
:102BD000F9CF81E001C085E0DF91CF911F910F9186
:102BE00008958093BA070C943A0881E09091BB074E
:102BF000911180E08093BB070E94A6068EEA92E0C6
:102C00000E9468068091BB07882319F08BEA92E046
:102C100002C087EA92E00E9468060E949F068091A7
:102C2000BB07882339F081E08093BA070E943A08F5
:102C30000C94AE0F0895CF93DF930E94A6068AE10D
:102C400093E00E9468060E94AE0F2AEE35E045E848
:102C500051E06FE375E187EB95E10E941A0810924D
:102C6000BB071092BC071092BA07C0E0D1E0809178
:102C7000EA07823051F50E946418C82F81FD25C0F3
:102C80000E9409158130C1F48091BA07811104C0F6
:102C900089E691E00E94D10E80916B01882339F37F
:102CA0008091BB07882329F0D093BA070E943A0885
:102CB000DECF1092BA07DBCF8823C9F28091BB0721
:102CC0008823A9F20E94F515D2CF60E081E00E942E
:102CD000F50F0E94A6068AE093E00E9468068C2FFA
:102CE000DF91CF910895CF93DF93EA018091BE07E2
:102CF00081FF1AC08D7F8093BE0765E871E080E197
:102D000091E00E94D90B6BE871E08FE697E00E949A
:102D1000D90B6FEF7FEF81E991E00E94FB0B8EE012
:102D200090E09983888310C0CA010E943F1380916C
:102D3000BE0782FF09C08B7F8093BE070E94A60654
:102D400089E393E00E9468061092BD0781E0DF915D
:102D5000CF9108958091BD0781110EC081E08093CD
:102D6000BD070E943A088091E907882379F00E9404
:102D7000A60683E393E008C08091E907882331F039
:102D80000E94A60689E293E00C94680608950F93CA
:102D90001F93CF93DF93EC018B010C960E94F30BF2
:102DA0008E3F2FEF920749F130F4039691F5809111
:102DB000BE0782603EC00E94A6068FE693E00E9496
:102DC00068068091BE0785608093BE072696BE0187
:102DD0008FE697E00E94A50C81112FC06FE677E087
:102DE000CE010E94D90B0E94920B0E94F71264E060
:102DF0008FE697E00E948D1220C00E94A6068DE506
:102E000093E00E9468068091BE078E7F8093BE0784
:102E100014C0C8010E9499138091BE0780FD0DC0A7
:102E20000E94A6068BE493E00E9468068091BE078C
:102E300086608093BE070E94AA1681E0DF91CF9141
:102E40001F910F910895DF92EF92FF920F931F93BE
:102E5000CF93DF9300D0CDB7DEB70E94A60685ECF6
:102E600093E00E9468062AEE35E045E851E067EC01
:102E700076E183E796E10E941A080E943313682FD7
:102E80008FE697E00E948D120E94AE0F1092BE074F
:102E90001092BD07D0907507FF24F39410E000E076
:102EA0008091EA07811155C00E946418082F81FDA6
:102EB00050C00E9409150E941813E82E882301F1C2
:102EC000FF2031F00E94A60683EB93E00E94680683
:102ED0008091BE0780FF03C00E94AA1610C0CE01D9
:102EE00001960E943F130E94A60684EA93E00E9486
:102EF000680689819A810E9419070E949F06F12C19
:102F0000DD2071F2112391F0E11021C060E080E03A
:102F10000E942A138091E907882331F00E94A606B7
:102F200089E993E00E94680610E0BACF81E08E152F
:102F3000D8F761E080E00E942A138091E907882396
:102F400031F00E94A6068FE893E00E94680611E027
:102F5000A7CF0E94E50F0E94F7120E94A60680E804
:102F600093E00E946806802F0F900F90DF91CF9121
:102F70001F910F91FF90EF90DF900895CF93DF9313
:102F8000EB0181E991E00E94F30B2091810721116F
:102F90000CC0039619F08FED93E00CC060E078E070
:102FA00081E991E00E94FB0B08C08115984029F04F
:102FB00083ED93E00E94680603C0CE010E9499133E
:102FC00081E0DF91CF9108952091BF073091C00734
:102FD000FA01318320836217730778F0209181070B
:102FE000211105C06DEF7FEF0C960E94FB0B109234
:102FF000C0071092BF0781E0089585E008951F93F0
:10300000CF93DF9300D0CDB7DEB70E94A6068EE047
:1030100094E00E9468062AEE35E045E851E06EEB48
:1030200077E184EE97E10E941A080E943313682F1B
:103030008FE697E00E948D120E94AE0F10E0809103
:10304000EA07813081F50E946418182F81FD2BC09A
:103050000E9409150E941813882389F3CE01019656
:103060000E943F138111EBCF89819A810E94EE1358
:103070008111E5CF89819A810E944C148823F9F24D
:103080002091BF073091C007232B21F080E094E00E
:103090000E94680629813A813093C0072093BF07B8
:1030A0000E943A08CCCF0E94E50F0E94F7120E94BE
:1030B000A6068CEE93E00E946806812F0F900F9079
:1030C000DF91CF911F910895AF92BF92CF92DF927F
:1030D000EF92FF920F931F93CF93DF930E943906D5
:1030E000811102C0F12C1CC10E9442068A3009F0F5
:1030F000E7C086EA94E00E946806E12CFF24F3947E
:1031000083EA94E00E946806C0E00E9442068A308A
:10311000C1F08F3711F0883031F4CC23B1F3C150B6
:103120000E946106F2CF90EE980F903670F7EC2F68
:10313000F0E0E753F84F80830E946106CF5FCF3104
:1031400021F70E949F06EC2FF0E0E753F84F108222
:10315000CC23B1F2D12C80E0A82FB0E0A753B84F18
:103160009C91903211F48F5FF7CF9923C9F0ED2D28
:10317000F0E0EE0FFF1FEF53F84FB183A083D3941D
:10318000E82FF0E0E753F84F90818F5F903221F005
:103190009111F6CF90E001C091E010829111DCCF47
:1031A000DD2009F480C00091C1071091C207F80129
:1031B00080818F3369F589E394E00E9468060CEF03
:1031C00014E0F80125913491A22EC22FD32F20971D
:1031D00009F469C0F8013496C590D490BC2EBA1891
:1031E000FE018491882321F00E9461062196F6CF8A
:1031F000F9E0FB1528F080E20E946106B394F8CF55
:10320000C6010E9468060E949F060A5F1F4FD9CF21
:10321000CCEFD4E0FE01659174916115710509F45C
:103220003EC0C8010E94F81A892B11F02696F2CFF1
:103230002097A9F12296FE012591349161EC77E067
:103240008D2DF9010995E82E0E9410070E94A30612
:103250008E2D807FB9F4F2E0EF1207C08BE994E085
:103260000E94680692E0F92E5BC083E0E81207C076
:1032700087E894E00E94680683E0F82E41CF82E858
:1032800094E00FC0803119F489E794E00AC08032DD
:1032900019F481E794E005C08BE694E002C084E66F
:1032A00094E00E946806E1E0EE122ACFFE1203C00D
:1032B0008EE594E002C089E494E00E94680630C084
:1032C0008F33D1F485E294E00E946806CCE1D7E028
:1032D000FE018491882311F13396059114910E9487
:1032E000610681E294E00E946806C8010E946806B7
:1032F0000E949F062596ECCFECE1F7E09491981799
:1033000029F0992309F4EECE3596F8CF309709F4D9
:10331000E9CE319685919491FC010995FF24F394AF
:103320008F2DDF91CF911F910F91FF90EF90DF9044
:10333000CF90BF90AF90089581E0089582E0089506
:10334000CF93DF9300D000D0CDB7DEB7FB01BE0135
:103350006F5F7F4F828193810E942E0C882341F002
:103360006BE777E0CE0101960E94E60B80E001C09A
:1033700081E10F900F900F900F90DF91CF91089502
:103380000F931F93CF93DF9300D0CDB7DEB7FB0130
:10339000A081B18111969C9111972C91243701F550
:1033A000903739F0943741F09C36D1F407E717E0B5
:1033B00005C00FE717E002C009E717E0813081F090
:1033C000BE016F5F7F4F828193810E9468058823D1
:1033D00039F089819A81F8019183808380E001C06E
:1033E00081E10F900F90DF91CF911F910F91089580
:1033F0000F931F93CF93DF9300D0CDB7DEB7FB01C0
:10340000A081B1812C9111969C91243741F49D3675
:1034100069F59091810720E001E817E011C0263698
:1034200029F5933641F0943609F59091760723E01B
:1034300006E717E005C09091750723E005E717E060
:10344000813021F4992371F080E00CC0BE016F5FE0
:103450007F4F828193812A830E9439052A818823A4
:1034600029F08981F8018083822F01C081E10F90CA
:103470000F90DF91CF911F910F910895CF93DF931C
:1034800000D000D000D0CDB7DEB7FB01BE016F5F2A
:103490007F4F828193810E945D0C882341F06FE60B
:1034A00077E0CE0101960E94D90B80E001C081E156
:1034B00026960FB6F894DEBF0FBECDBFDF91CF9139
:1034C00008950E94AE0F80E008950E94E50F80E00D
:1034D00008950E94A70B80E008950E94B30B8823F3
:1034E00011F08062089580E008950E94920B882375
:1034F00011F08062089580E008950E942E0B80E014
:1035000008958DEE94E00E94680680E0089582E0C0
:103510008093EA07089583E08093EA070895109264
:10352000EA07089581E08093EA0708950C94F51561
:1035300081E00C94F11580E00C94F11581E09091FC
:10354000E907911180E08093E90782E197E00E940A
:1035500068068091E907882319F08DE097E002C0A2
:1035600087E097E00C9468060C94AE0F0C94E50F7E
:103570000E948E040E942B070E94FB050E94E50713
:103580008AEB98E00E9468068EE898E00E94680640
:103590000E94D30B0E942E0B0E949F0683E598E0A9
:1035A0000E9468068091EA07823039F0833041F04A
:1035B000813049F40E94FF1708C00E941B1605C005
:1035C0000E94B11402C00E942317823059F784E48C
:1035D00098E00E9468062FEF81EE94E02150804031
:1035E0009040E1F700C00000C3CFF8940C947C1B1E
:1035F000FB01DC018D91059080190110D9F3990B25
:103600000895DC01CB01FC01F999FECF06C0F2BDA3
:10361000E1BDF89A319600B40D9241505040B8F790
:103620000895A8E1B0E042E050E00C94031BDC01F7
:10363000CB0103C02D910E94221B41505040D0F776
:103640000895262FF999FECF1FBA92BD81BD20BDE6
:103650000FB6F894FA9AF99A0FBE019608950E944F
:10366000211B272F0C94221B991B79E004C0991F62
:10367000961708F0961B881F7A95C9F780950895CC
:10368000A1E21A2EAA1BBB1BFD010DC0AA1FBB1F66
:10369000EE1FFF1FA217B307E407F50720F0A21BD8
:1036A000B30BE40BF50B661F771F881F991F1A9445
:1036B00069F760957095809590959B01AC01BD016F
:1036C000CF0108950E946D1BA59F900DB49F900D92
:1036D000A49F800D911D11240895A29FB001B39F56
:1036E000C001A39F700D811D1124911DB29F700D0B
:0C36F000811D1124911D0895F894FFCF56
:1036FC008813FFFFFFFF0000000000000000000027
:10370C00FFFFFFFFFFFFBB01B101B401B10130307E
:10371C003A30303A30303A30303A30303A3030009B
:10372C003030302E3030302E3030302E30303000C3
:00000001FF
